:1000000012C02CC02BC02AC029C028C027C026C0BF
:1000100025C024C023C022C021C020C01FC01EC0D4
:100020001DC01CC01BC011241FBECFE5D4E0DEBF25
:10003000CDBF10E0A0E6B0E0ECE8F1E002C0059032
:100040000D92A036B107D9F710E0A0E6B0E001C0EC
:100050001D92A036B107E1F76DD097C0D1CFCF93F5
:10006000DF93CDB7DEB7E8E3F0E01082E5E3F0E040
:1000700080E28083E2E3F0E01082E7E3F0E01082C8
:10008000E4E3F0E080E28083E1E3F0E01082EBE57E
:10009000F0E01082E5E5F0E01082DF91CF91089565
:1000A000CF93DF93CDB7DEB723970FB6F894DEBFBB
:1000B0000FBECDBF89838981282F33273B832A83B5
:1000C0008A819B81009731F02A813B812130310563
:1000D00049F010C0A5E3B0E0E5E3F0E080818F7D5A
:1000E0008C931FC0A5E3B0E0E5E3F0E0808180627F
:1000F0008C9317C0E5E3F0E08081992780729070BF
:10010000009741F0A5E3B0E0E5E3F0E080818F7D6A
:100110008C9307C0A5E3B0E0E5E3F0E08081806266
:100120008C9323960FB6F894DEBF0FBECDBFDF9140
:10013000CF910895CF93DF93CDB7DEB722970FB657
:10014000F894DEBF0FBECDBF8ADF00C0E0E3F0E071
:1001500080819927847090700097C1F780E0A0DFBC
:100160008FEF9FEF9A83898305C089819A810197D8
:100170009A83898389819A810097B9F700000000EA
:0C0180000000000081E08CDFE1CFFFCF29
:00000001FF
